:020000040800F2
:1000000000060020E1010008610E0008E10D000873
:10001000390E0008E10D00080D0E0008E30100088C
:10002000E3010008E3010008E3010008C120000823
:10003000E3010008E3010008E3010008E301000810
:10004000E3010008E3010008E3010008E301000800
:10005000E3010008E301000889310008B531000818
:10006000E13100080D32000839320008E3010008D0
:10007000E3010008E3010008E3010008E3010008D0
:10008000E3010008E3010008E3010008E3010008C0
:10009000E3010008E3010008E301000865320008FD
:1000A000E3010008E3010008E3010008E3010008A0
:1000B000FD2F0008E3010008E3010008E301000848
:1000C000E3010008E3010008E3010008E301000880
:1000D000E3010008E3010008E3010008E301000870
:1000E000CD320008E3010008E3010008E301000845
:1000F000E3010008E3010008E3010008E301000850
:10010000E3010008E3010008E3010008E30100083F
:10011000E3010008E3010008E3010008E30100082F
:10012000E3010008E3010008E3010008E30100081F
:10013000E3010008E3010008E3010008E30100080F
:10014000E3010008E3010008E3010008F9270008C3
:10015000E3010008E3010008E3010008E3010008EF
:10016000E3010008E3010008E3010008E3010008DF
:10017000E3010008E3010008E3010008E3010008CF
:10018000E3010008E3010008E3010008E3010008BF
:10019000E3010008E3010008E3010008E3010008AF
:1001A000E3010008E3010008E3010008E30100089F
:1001B000E3010008E3010008E3010008E30100088F
:1001C000E3010008E3010008E3010008E30100087F
:1001D000E3010008E3010008E3010008E30100086F
:1001E00002E000F000F8FEE772B63A4880F30888B3
:1001F000394880F3098839484EF60851CEF200019B
:10020000086040F20000CCF200004EF63471CEF2ED
:1002100000010860BFF34F8FBFF36F8F40F2000003
:10022000C0F2F0004EF68851CEF200010860BFF334
:100230004F8FBFF36F8F4FF00000E1EE100A4EF6C4
:100240003C71CEF200010860062080F31488BFF3F1
:100250006F8F01F0B5FF01F091FF02F033FE4FF018
:1002600055301F491B4A91423CBF41F8040BFAE745
:100270001C49194A91423CBF41F8040BFAE71A495C
:100280001A4A1B4B9A423EBF51F8040B42F8040B2A
:10029000F8E700201749184A91423CBF41F8040B87
:1002A000FAE701F06FFF02F061FE144C144DAC420E
:1002B00003DA54F8041B8847F9E700F041F8114CC1
:1002C000114DAC4203DA54F8041B8847F9E701F0FA
:1002D00057BF000000060020002200200000000898
:1002E0000000002000060020F83600080022002050
:1002F0004022002040220020A42D0020E001000820
:10030000E0010008E0010008E00100082DE9F04FDD
:100310002DED108AC1F80CD0C3689D46BDEC108A43
:10032000BDE8F08F002383F311882846A047002002
:1003300001F0E8FAFEE701F07DFA00DFFEE70000D9
:1003400038B501F08FFE054601F0B4FE0446D8B979
:100350000F4B9D421AD001339D4218BF044641F213
:10036000883504BF01240025002001F085FE0CB172
:1003700000F056F800F00AFD00F086FB284600F079
:10038000A7F800F04DF8F9E70025EDE70546EBE7A3
:10039000010007B008B500F049FBA0F12003584266
:1003A000584108BD07B541F21203022101A8ADF87A
:1003B000043000F059FB03B05DF804FB10B52023B6
:1003C00083F311881248C3680BB101F021FB114A75
:1003D0000F4800234FF47A7101F0DEFA002383F313
:1003E00011880D4C236813B12368013B23606368B7
:1003F00013B16368013B6360084B1B7833B96368D2
:1004000023B9022000F034FC3223636010BD00BF2A
:1004100040220020BD0300085C230020542200205D
:10042000254B264A10B51C461968013142D00433C9
:100430009342F9D16268224B9A423BD9214B9B6887
:1004400003F1006303F580339A4233D2002000F0B9
:1004500035FB1D4B0220187000F0FCFB1B4B1A6C87
:1004600000221A64196E1A66196E596C5A64596E14
:100470005A665A6E5A6942F080025A615A6922F0ED
:1004800080025A615A691A6942F000521A611A6967
:1004900022F000521A611B6972B64FF0E02320214E
:1004A000C3F8084DD4E9003281F311889D4683F3E7
:1004B0000888104710BD00BF000001082000010897
:1004C000FFFF0008002200205422002000380240D4
:1004D0002DE9F04F93B0A94B00902022FF210AA8EC
:1004E0009D6800F0FDFBA64A1378A3B9A548012139
:1004F000C3601170202383F31188C3680BB101F02E
:1005000087FAA14A9F4800234FF47A7101F044FA18
:10051000002383F31188009B9C4A03B113609C491C
:10052000009C00230B70536098469B461E469A46DB
:10053000012000F08FFB24B1944B1B68002B00F0CE
:100540001682002000F072FA0390039B002BF2DB6E
:10055000012000F06FFB039B213B162BE8D801A282
:1005600052F823F0C1050008E90500087D060008DF
:1005700031050008310500083105000811070008A1
:10058000E3080008FD0700085F0800088708000866
:10059000AD08000831050008BF0800083105000853
:1005A00031090008610600083105000875090008D6
:1005B000CD05000861060008310500085F08000845
:1005C0000220FFF7E7FE002840F0FB81009B02219C
:1005D000B8F1000F08BF1C4605A841F21233ADF870
:1005E000143000F041FAA3E74FF47A7000F01EFADD
:1005F000071EEBDB0220FFF7CDFE0028E6D0013F0F
:10060000052F00F2E081DFE807F0030A0D10133632
:1006100005230593042105A800F026FA17E05748A2
:100620000421F9E75B480421F6E75B480421F3E77E
:100630004FF01C09484600F043FA09F104090590FF
:10064000042105A800F010FAB9F12C0FF2D1012015
:1006500000FA07F747EA0B0B5FFA8BFB4FF0000A33
:1006600000F08AFB26B10BF00B030B2B08BF002414
:10067000FFF798FE5CE749480421CDE7002EA5D09E
:100680000BF00B030B2BA1D10220FFF783FE0746D3
:1006900000289BD001203E4E00F010FA022030705E
:1006A00000F0D8FA4FF000085FFA88F9484600F0E9
:1006B00015FA044690B1484600F020FA08F1010806
:1006C0000028F1D1B846044641F21213022105A8D0
:1006D000ADF814303E4600F0C7F929E701230220A7
:1006E000337000F0A7FA2546244B9B68AB4207D92C
:1006F000284600F0E5F9013040F068810435F3E761
:10070000234B00251D70214BB8465D603E46A7E790
:10071000002E3FF45BAF0BF00B030B2B7FF456AFB7
:100720001B4B0220187000F095FA322000F07EF981
:10073000B0F10009FFF64AAF19F003077FF446AFA6
:100740000E4A926809EB050393423FF63FAFB9F5B5
:10075000807F3FF73BAF124B0193B94522DD4FF449
:100760007A7000F063F90390039A002AFFF62EAF27
:10077000019B039A03F8012B0137EDE700220020CB
:100780005823002040220020BD0300085C230020E5
:100790005422002004220020082200200C220020E5
:1007A00058220020C820FFF7F5FD074600283FF437
:1007B0000DAF1F2D11D8C5F120024A450AAB25F017
:1007C000030028BF4A4683490192184400F062FAA8
:1007D000019A8048FF2100F083FA4FEAA9037D497E
:1007E0000193C9F38702284600F082FA06460028E2
:1007F0003FF46AAF019B05EB830531E70220FFF769
:10080000C9FD00283FF4E2AE00F0A2F900283FF451
:10081000DDAE0027B946704B9B68BB4218D91F2F2D
:1008200011D80A9B01330ED027F0030312AA1344F8
:1008300053F8203C05934846042205A900F012FB1A
:1008400004378146E7E7384600F03AF90590F2E7C9
:10085000CDF81490042105A800F006F900E7002364
:10086000642104A8049300F0F5F800287FF4AEAEEC
:100870000220FFF78FFD00283FF4A8AE049800F097
:100880004FF90590E6E70023642104A8049300F0E3
:10089000E1F800287FF49AAE0220FFF77BFD0028E4
:1008A0003FF494AE049800F04BF9EAE70220FFF71A
:1008B00071FD00283FF48AAE00F05AF9E1E702200A
:1008C000FFF768FD00283FF481AE05A9142000F071
:1008D00055F904210746049004A800F0C5F83946EC
:1008E000B9E7322000F0A2F8071EFFF66FAEBB0793
:1008F0007FF46CAE384A926807EB0A0393423FF6E6
:1009000065AE0220FFF746FD00283FF45FAE27F0FA
:1009100003075744BA453FF4A3AE504600F0D0F861
:100920000421059005A800F09FF80AF1040AF1E7F8
:100930004FF47A70FFF72EFD00283FF447AE00F029
:1009400007F9002844D00A9B01330BD008220AA9DA
:10095000002000F0CDF900283AD02022FF210AA87B
:1009600000F0BEF9FFF71EFD1C4800F0D1FF13B0E8
:10097000BDE8F08F002E3FF429AE0BF00B030B2BDC
:100980007FF424AE0023642105A8059300F062F8EB
:10099000074600287FF41AAE0220FFF7FBFC8146D1
:1009A00000283FF413AEFFF7FDFC41F2883000F061
:1009B000AFFF059800F012FA4E4600F0DDF93C4614
:1009C000B6E506464CE64FF0000AFFE5B8467BE682
:1009D000374679E65822002000220020A086010038
:1009E00070B50F4B1B780133DBB2012B0C4611D8CD
:1009F0000C4D29684FF47A730E6AA2FB033201464C
:100A000022462846B047844204D1074B00221A7080
:100A1000012070BD4FF4FA7000F07AFF0020F8E773
:100A200010220020502500209023002007B500232D
:100A3000024601210DF107008DF80730FFF7D0FFC6
:100A400020B19DF8070003B05DF804FB4FF0FF30C4
:100A5000F9E700000A4608B50421FFF7C1FF80F05E
:100A60000100C0B2404208BD30B4054C2368DD69C6
:100A7000044B0A46AC460146204630BC604700BFE6
:100A800050250020A086010070B501F0F1F9094E53
:100A9000094D3080002428683388834208D901F04A
:100AA000E1F92B6804440133B4F5803F2B60F2D3A5
:100AB00070BD00BF922300206423002001F086BA9D
:100AC00000F1006000F580300068704700F10060C0
:100AD000920000F5803001F011BA0000054B1A6851
:100AE000054B1B889B1A834202D9104401F0BAB906
:100AF00000207047642300209223002038B5074D62
:100B000004462868204401F0B5F928B92868204433
:100B1000BDE8384001F0C6B938BD00BF64230020ED
:100B200010F003030AD1B0F5047F05D200F10050A4
:100B3000A0F51040D0F80038184670470023FBE7B6
:100B400000F10050A0F51040D0F8100A70470000E6
:100B5000064991F8243033B10023086A81F8243023
:100B60000822FFF7B3BF0120704700BF68230020B1
:100B7000014B1868704700BF002004E070B52A4B95
:100B80001B68C3F30B0204461B0C62B140F2134016
:100B9000824230D040F2194082422ED040F22140B1
:100BA00082422CD10322214D0C2000FB02525568B9
:100BB00042F20102934224D0B3F5805F23D041F288
:100BC0000102934221D041F2030293421FD041F22D
:100BD0000702934214BF3F233123013C0C44013DE3
:100BE0000A46A24215D215F9016F501C9EB100F8B9
:100BF000016C0246F5E70122D5E70222D3E70C4D4E
:100C0000D6E73323E9E74123E7E75A23E5E759230A
:100C1000E3E7104605E02C258442157001D9901CAD
:100C20005370401A70BD00BF002004E0F833000884
:100C3000CC330008022804D1054B4FF400129A610E
:100C400070470128FCD1024B4FF48012F7E700BF38
:100C500000040240022803D1044B20229A6170470D
:100C60000128FCD1014B1022F8E700BF000402402C
:100C7000022805D1064A536983F020035361704767
:100C80000128FCD1024A536983F01003F6E700BF44
:100C90000004024010B50023934203D0CC5CC4543E
:100CA0000133F9E710BD000010B5013810F9013F1C
:100CB0003BB191F900409C4203D11AB10131013A94
:100CC000F4E71AB191F90020981A10BD1046FCE71C
:100CD00003460246D01A12F9011B0029FAD17047C7
:100CE00002440346934202D003F8011BFAE770471F
:100CF0002DE9F8431F4D144695F8242007468846F1
:100D000052BBDFF870909CB395F824302BB92022A9
:100D1000FF2148462F62FFF7E3FF95F82400C0F15A
:100D20000802A24228BF2246D6B24146920005EBF5
:100D30008000FFF7AFFF95F82430A41B1E44F6B2E5
:100D4000082E17449044E4B285F82460DBD1FFF705
:100D5000FFFE0028D7D108E02B6A03EB8203834211
:100D6000CFD0FFF7F5FE0028CBD10020BDE8F883F7
:100D70000120FBE768230020024B1A78024B1A700F
:100D8000704700BF902300201022002010B50F4CA8
:100D90000F4800F0F7F821460D4800F01FF92468CD
:100DA0000C48626DD2F8043843F00203C2F80438EC
:100DB00000F0AEFD0849204600F016FA626DD2F848
:100DC000043823F00203C2F8043810BDEC340008E4
:100DD0005025002040420F00F43400087047000006
:100DE00000B59BB0EFF3098168226846FFF752FF18
:100DF000EFF30583044B9A6BDA6A9A6A9A6A9A6AE5
:100E00009A6A9A6A9B6AFEE700ED00E000B59BB023
:100E1000EFF3098168226846FFF73CFFEFF3058393
:100E2000044B9A6B9A6A9A6A9A6A9A6A9A6A9B6A55
:100E3000FEE700BF00ED00E000B59BB0EFF30981D5
:100E400068226846FFF726FFEFF30583034B5A6BD2
:100E50009A6A9A6A9A6A9A6A9B6AFEE700ED00E0CB
:100E6000FEE7000030B5094D0A4491420DD011F85B
:100E7000013B5840082340F30004013B2C4013F091
:100E8000FF0384EA5000F6D1EFE730BD2083B8EDD0
:100E9000026843681143016003B1184770470000BE
:100EA00013B5446BD4F894341A681178042915D119
:100EB000217C022912D11979128901238B40134216
:100EC0000CD101A904F14C0001F002FFD4F89444C4
:100ED000019B21790246206800F0CEF902B010BDD6
:100EE000143001F085BE00004FF0FF33143001F0E4
:100EF0007FBE00004C3001F057BF00004FF0FF33C1
:100F00004C3001F051BF0000143001F053BE00001E
:100F10004FF0FF31143001F04DBE00004C3001F0B5
:100F200023BF00004FF0FF324C3001F01DBF000026
:100F30000020704710B5D0F894341A68117804294D
:100F4000044617D1017C022914D159795289012311
:100F50008B4013420ED1143001F0E6FD024648B139
:100F6000D4F894444FF4807361792068BDE8104050
:100F700000F070B910BD0000406BFFF7DBBF000050
:100F8000704700007FB5124B036000234360C0E947
:100F90000233012502260F4B05740446029001938B
:100FA00000F18402294600964FF48073143001F05A
:100FB00097FD094B0294CDE9006304F523724FF4C9
:100FC0008073294604F14C0001F05EFE04B070BD50
:100FD00028340008790F0008A10E00080B682022B1
:100FE00082F311880A7903EB820290614A7909320F
:100FF00043F822008A7912B103EB8203986102233D
:101000000374C0F89414002383F311887047000020
:1010100038B5037F044613B190F85430ABB9201DA6
:1010200001250221FFF734FF04F1140025776FF04A
:10103000010100F095FC84F8545004F14C006FF06D
:101040000101BDE8384000F08BBC38BD10B501216E
:1010500004460430FFF71CFF0023237784F8543044
:1010600010BD000038B504460025143001F050FDD5
:1010700004F14C00257701F01FFE201D84F8545028
:101080000121FFF705FF2046BDE83840FFF752BFBA
:1010900090F8443003F06003202B07D190F84520EE
:1010A000212A4FF0000303D81F2A06D800207047DA
:1010B000222AFBD1C0E90E3303E0034A82630722F0
:1010C000C2630364012070471122002037B5D0F8B5
:1010D00094341A681178042904461AD1017C022933
:1010E00017D11979128901238B40134211D100F1D4
:1010F0004C05284601F0A0FE58B101A9284601F090
:10110000E7FDD4F89444019B21790246206800F061
:10111000B3F803B030BD0000F0B500EB810385B03B
:101120009E6904460D46FEB1202383F3118804EB2B
:101130008507301D0821FFF7ABFEFB685B691B6864
:1011400006F14C001BB1019001F0D0FD019803A9FC
:1011500001F0BEFD024648B1039B2946204600F03F
:101160008BF8002383F3118805B0F0BDFB685A6942
:101170001268002AF5D01B8A013B1340F1D104F11B
:101180004402EAE7093138B550F82140DCB12023A8
:1011900083F31188D4F894241368527903EB820303
:1011A000DB689B695D6845B104216018FFF770FE3C
:1011B000294604F1140001F0C1FC2046FFF7BAFEF5
:1011C000002383F3118838BD7047000001F06EB82A
:1011D000012303700023C0E90133C361836203620A
:1011E000C36243620363704738B50446202383F328
:1011F00011880025C0E90355C0E90555416001F09B
:1012000065F80223237085F3118838BD70B500EBB3
:10121000810305465069DA600E46144618B1102263
:101220000021FFF75DFDA06918B110220021FFF732
:1012300057FD31462846BDE8704001F011B9000065
:10124000826802F0011282600022C0E904228261F9
:1012500001F092B9F0B400EB81044789E4680125FC
:10126000A4698D403D43458123600023A2606360F3
:10127000F0BC01F0ADB90000F0B400EB81040789C7
:10128000E468012564698D403D43058123600023A6
:10129000A2606360F0BC01F027BA000070B50223C1
:1012A000002504460370C0E90255C0E90455C56431
:1012B000856180F8345001F06FF863681B6823B1D2
:1012C00029462046BDE87040184770BD037880F875
:1012D00050300523037043681B6810B504460BB1FA
:1012E000042198470023A36010BD000090F850200F
:1012F000436802701B680BB1052118477047000056
:1013000070B590F83430044613B1002380F83430BF
:1013100004F14402204601F051F963689B68B3B9B7
:1013200094F8443013F0600535D00021204601F0D8
:10133000A3FB0021204601F095FB63681B6813B1F5
:10134000062120469847062384F8343070BD204695
:1013500098470028E4D0B4F84A30E26B9A4288BF3C
:10136000E36394F94430E56B002B4FF0200380F2E7
:101370000381002D00F0F280092284F8342083F3E9
:1013800011880021D4E90E232046FFF775FF0023C2
:1013900083F31188DAE794F8452003F07F0343EAEA
:1013A000022340F20232934200F0C58021D8B3F507
:1013B000807F48D00DD8012B3FD0022B00F09380C6
:1013C000002BB2D104F14C02A2630222E263236437
:1013D000C1E7B3F5817F00F09B80B3F5407FA4D1D6
:1013E00094F84630012BA0D1B4F84C3043F00203FE
:1013F00032E0B3F5006F4DD017D8B3F5A06F31D000
:10140000A3F5C063012B90D8636894F846205E680A
:1014100094F84710B4F848302046B047002884D0EC
:101420004368A3630368E3631AE0B3F5106F36D033
:1014300040F6024293427FF478AF5C4BA3630223F1
:10144000E3630023C3E794F84630012B7FF46DAFCC
:10145000B4F84C3023F00203C4E90E55A4F84C3024
:10146000256478E7B4F84430B3F5A06F0ED194F852
:10147000463084F84E30204600F0E6FF63681B6873
:1014800013B1012120469847032323700023C4E9A8
:101490000E339CE704F14F03A3630123C3E72378D2
:1014A000042B10D1202383F311882046FFF7C8FEB8
:1014B00085F311880321636884F84F5021701B68FD
:1014C0000BB12046984794F84630002BDED084F8C4
:1014D0004F300423237063681B68002BD6D0022191
:1014E00020469847D2E794F848301D0603F00F01D4
:1014F00020460AD501F054F8012804D002287FF4D0
:1015000014AF2B4B9AE72B4B98E701F03BF8F3E72E
:1015100094F84630002B7FF408AF94F8483013F06D
:101520000F01B3D01A06204602D501F0B9FAADE793
:1015300001F0ACFAAAE794F84630002B7FF4F5AE40
:1015400094F8483013F00F01A0D01B06204602D5B6
:1015500001F092FA9AE701F085FA97E7142284F8ED
:10156000342083F311882B462A4629462046FFF76C
:1015700071FE85F31188E9E65DB1152284F8342007
:1015800083F311880021D4E90E232046FFF762FE81
:10159000FDE60B2284F8342083F311882B462A467B
:1015A00029462046FFF768FEE3E700BF58340008ED
:1015B000503400085434000838B590F834300446EC
:1015C000002B3ED0063BDAB20F2A34D80F2B32D88C
:1015D000DFE803F037313108223231313131313136
:1015E00031313737C56BB0F84A309D4214D2C368E9
:1015F0001B8AB5FBF3F203FB12556DB9202383F36D
:1016000011882B462A462946FFF736FE85F31188B6
:101610000A2384F834300EE0142384F83430202375
:1016200083F3118800231A4619462046FFF712FE5D
:10163000002383F3118838BD036C03B1984700235E
:10164000E7E70021204601F017FA0021204601F0CB
:1016500009FA63681B6813B10621204698470623E0
:10166000D7E7000010B590F83430142B044629D089
:1016700017D8062B05D001D81BB110BD093B022B92
:10168000FBD80021204601F0F7F90021204601F0A7
:10169000E9F963681B6813B10621204698470623C1
:1016A00019E0152BE9D10B2380F83430202383F384
:1016B000118800231A461946FFF7DEFD002383F345
:1016C0001188DAE7C3689B695B68002BD5D1036C8E
:1016D00003B19847002384F83430CEE7024B002250
:1016E000C3E900339A6070479423002000230374F9
:1016F0008268054B1B6899689142FBD25A68036067
:1017000042601060586070479423002008B5202381
:1017100083F31188037C032B05D0042B0DD02BB948
:1017200083F3118808BD436900221A604FF0FF332C
:101730004361FFF7DBFF0023F2E7D0E900321360DB
:101740005A60F3E7002303748268054B1B689968AD
:101750009142FBD85A68036042601060586070473D
:1017600094230020054B19690874186802681A60F0
:101770005360186101230374FEF7C8BD9423002051
:1017800030B54B1C0B4D87B0044610D02B690A4A6C
:1017900001A800F001F92046FFF7E4FF049B13B114
:1017A00001A800F035F92B69586907B030BDFFF783
:1017B000D9FFF8E7942300200D17000838B50C4D29
:1017C00041612B6981689A689142044603D8BDE85B
:1017D0003840FFF78BBF1846FFF7B4FF01232C6199
:1017E000014623742046BDE83840FEF78FBD00BF98
:1017F00094230020044B1A681B6990689B689842E8
:1018000094BF0020012070479423002010B5084C9D
:10181000236820691A6822605460012223611A74C7
:10182000FFF790FF01462069BDE81040FEF76EBD4E
:1018300094230020FFF7EABFFEE7000010B50C4C30
:10184000FFF74CFF00F09AF80A498022204600F08A
:1018500021F8012344F8180C037400F041FC002324
:1018600083F3118862B60448BDE8104000F032B836
:10187000BC2300205C3400086C34000800F002B97E
:10188000034A516853685B1A9842FBD8704700BFFF
:10189000001000E082600222028270478368A3F198
:1018A0007C0243F80C2C026943F83C2C426943F853
:1018B000382C074A43F81C2CC26843F8102C02222B
:1018C00003F8082C002203F8072CA3F11800704736
:1018D0002503000810B5202383F31188FFF7DEFFEE
:1018E00000210446FFF76AFF002383F31188204696
:1018F00010BD0000024B1B6958610F20FFF732BF7B
:1019000094230020202383F31188FFF7F3BF000006
:1019100008B50146202383F311880820FFF730FF24
:10192000002383F3118808BD49B1064B42681B6947
:1019300018605A60136043600420FFF721BF4FF026
:10194000FF307047942300200368984206D01A683D
:101950000260506059611846FFF7C8BE704700002A
:1019600038B504460D462068844200D138BD03686E
:1019700023605C604561FFF7B9FEF4E7054B03F1B6
:101980001402C3E905224FF0FF310022C3E9071218
:10199000704700BF9423002070B51C4EC0E903239C
:1019A00005460C4601F07AFA334653F8142F9A4252
:1019B0000DD13062C5E901242A600A2C2CBF001920
:1019C0000A30C6E90555BDE8704001F055BA316AE4
:1019D000431AE31838BF1C469368A34202D908197A
:1019E00001F058FA73699A6894420CD85A68AC604E
:1019F0002B606A6015609A685D60121B9A604FF0F8
:101A0000FF33F36170BD1B68A41AECE79423002038
:101A100038B51B4C636998420DD0D0E90032136091
:101A20005A6000228168C2609A680A449A604FF046
:101A3000FF33E36138BD2246036842F8143F0021BA
:101A400093425A60C16003D1BDE8384001F01CBA2E
:101A50009A688168256A0A449A6001F01FFA6369EE
:101A60009A68411B8A42E5D9AB181D1A092D206AD4
:101A700098BF01F10A02BDE83840104401F00ABAEB
:101A8000942300202DE9F041184C002704F114069E
:101A9000656901F003FA236AAA68C11A8A4215D857
:101AA00013442362D5E9003213605A606369D5F8A4
:101AB0000C80EF60B34201D101F0E6F987F31188A1
:101AC0002869C047202383F31188E1E76169B142A7
:101AD00009D013441B1ABDE8F0410A2B2CBFC018D3
:101AE0000A3001F0D7B9BDE8F08100BF942300208F
:101AF00000207047FEE70000704700004FF0FF3005
:101B00007047000002290CD0032904D0012907489E
:101B100018BF00207047032A05D8054800EBC20013
:101B20007047044870470020704700BF50350008D8
:101B3000202200200435000870B59AB005460846FA
:101B400001A9144600F0C2F801A8FFF7C1F8431C30
:101B50005B00C5E900340022237003236370C6B222
:101B600001AB02341046D1B28E4204F1020401D816
:101B70001AB070BD13F8011B04F8021C04F8010C24
:101B80000132F0E708B5202383F311880348FFF7FB
:101B90009DFA002383F3118808BD00BF5025002063
:101BA00090F8443003F01F02012A07D190F8452035
:101BB0000B2A03D10023C0E90E3315E003F06003C4
:101BC000202B08D1B0F848302BB990F84520212AB5
:101BD00003D81F2A04D8FFF75BBA222AEBD0FAE712
:101BE000034A82630722C26303640120704700BF77
:101BF0001822002007B5052917D8DFE801F01916CB
:101C000003191920202383F31188104A0190012120
:101C1000FFF7FCFA01980E4A0221FFF7F7FA0D4888
:101C2000FFF720FA002383F3118803B05DF804FB6B
:101C3000202383F311880748FFF7EAF9F2E720230E
:101C400083F311880348FFF701FAEBE7A434000897
:101C5000C83400085025002038B50C4D0C4C0D49F7
:101C60002A4604F10800FFF767FF05F1CA0204F1F4
:101C700010000949FFF760FF05F5CA7204F118006A
:101C80000649BDE83840FFF757BF00BF182A0020BB
:101C900020220020843400088E3400089934000883
:101CA00070B5044608460D46FFF712F8C6B2204646
:101CB000013403780BB9184670BD32462946FEF749
:101CC000F3FF0028F3D10120F6E700002DE9F84FDB
:101CD00005460C46FEF7FCFF2B49C6B22846FFF727
:101CE000DFFF08B10536F6B228492846FFF7D8FFCE
:101CF00008B11036F6B2632E0DD8DFF88C80DFF80D
:101D00008C90234FDFF890A0DFF890B02E7846B982
:101D10002670BDE8F88F29462046BDE8F84F01F04F
:101D20004DBB252E2BD1072241462846FEF7BCFF8E
:101D300058B9DBF800302360DBF804306360DBF86F
:101D40000830A36007350C34E0E7082249462846EE
:101D5000FEF7AAFF98B90F4BA21C197809090232A5
:101D6000C95D02F8041C13F8011B01F00F01534573
:101D7000C95D02F8031CF0D118340835C6E704F831
:101D8000016B0135C2E700BF7035000899340008C7
:101D900085350008107AFF1F1C7AFF1F7835000870
:101DA000BFF34F8F024AD368DB03FCD4704700BFF8
:101DB000003C024008B5094B1B7873B9FFF7F0FFF0
:101DC000074B1A69002ABFBF064A5A6002F18832DF
:101DD0005A601A6822F480621A6008BD762C0020CE
:101DE000003C02402301674508B50B4B1B7893B9B3
:101DF000FFF7D6FF094B1A6942F000421A611A68D0
:101E000042F480521A601A6822F480521A601A68EA
:101E100042F480621A6008BD762C0020003C02402B
:101E20000B28F0B516D80C4C0C4923787BB90C4D17
:101E30000E460C234FF0006255F8047B46F8042B45
:101E4000013B13F0FF033A44F6D10123237051F80C
:101E50002000F0BD0020FCE7A82C0020782C0020FA
:101E600098350008014B53F820007047983500085A
:101E70000C2070470B2810B5044601D9002010BD76
:101E8000FFF7CEFF064B53F824301844C21A0BB9A3
:101E90000120F4E712680132F0D1043BF6E700BFFD
:101EA000983500080B2810B5044621D8FFF778FFB5
:101EB000FFF780FF0F4AF323D360C300DBB243F484
:101EC000007343F002031361136943F48033136119
:101ED000FFF766FFFFF7A4FF074B53F8241000F04D
:101EE000D9F8FFF781FF2046BDE81040FFF7C2BFD9
:101EF000002010BD003C024098350008F8B512F0F3
:101F00000103144642D18218B2F1016F57D82D4B0C
:101F10001B6813F0010352D02B4DFFF74BFFF32347
:101F2000EB60FFF73DFF40F20127032C15D824F0AA
:101F300001046618244C401A40F20117B14223698B
:101F400000EB010524D123F001032361FFF74CFFCF
:101F50000120F8BD043C0430E7E78307E7D12B6993
:101F600023F440732B612B693B432B6151F8046BC5
:101F70000660BFF34F8FFFF713FF03689E42E9D05F
:101F80002B6923F001032B61FFF72EFF0020E0E710
:101F900023F44073236123693B4323610B882B8027
:101FA000BFF34F8FFFF7FCFE2D8831F8023BADB237
:101FB000AB42C3D0236923F001032361E4E7184651
:101FC000C7E700BF00380240003C0240084908B59E
:101FD0000B7828B11BB9FFF7EDFE01230B7008BD8C
:101FE000002BFCD0BDE808400870FFF7FDBE00BF25
:101FF000762C002010B50244064BD2B2904200D19C
:1020000010BD441C00B253F8200041F8040BE0B2AC
:10201000F4E700BF502800400F4B30B51C6F24047C
:1020200007D41C6F44F400741C671C6F44F4004414
:102030001C670A4C236843F4807323600244084BF6
:10204000D2B2904200D130BD441C00B251F8045BC2
:1020500043F82050E0B2F4E700380240007000403E
:102060005028004007B5012201A90020FFF7C2FF58
:10207000019803B05DF804FB13B50446FFF7F2FFC7
:10208000A04205D0012201A900200194FFF7C4FF5E
:1020900002B010BD70470000044BD3F874389B00A9
:1020A00042BF034B01221A70704700BF003002404C
:1020B000A92C0020014B1878704700BFA92C0020E4
:1020C000EFF3098305494A6B22F001024A63683342
:1020D00083F30988002383F31188704700EF00E041
:1020E000202080F3118862B60C4B0D4AD96821F488
:1020F000E0610904090C0A43DA60D3F8FC200949BD
:1021000042F08072C3F8FC200A6842F001020A60C3
:102110001022DA7783F82200704700BF00ED00E05C
:102120000003FA05001000E010B5202383F31188A6
:102130000E4B5B6813F4006314D0F1EE103AEFF32A
:102140000984683C4FF08073E361094BDB6B2366C5
:1021500084F30988FFF74EFB10B1064BA36110BD55
:10216000054BFBE783F31188F9E700BF00ED00E0C2
:1021700000EF00E0370300083A0300087047000052
:10218000FEE700000A4B0B480B4A90420BD30B4B67
:10219000DA1C121AC11E22F003028B4238BF002241
:1021A0000021FEF79DBD53F8041B40F8041BECE72B
:1021B00038370008A42D0020A42D0020A42D0020D5
:1021C0007047000070B5D0E915439E6800224FF0BB
:1021D000FF3504EB42135101D3F800090028BEBFBC
:1021E000D3F8000940F08040C3F80009D3F8000B91
:1021F0000028BEBFD3F8000B40F08040C3F8000BAE
:10220000013263189642C3F80859C3F8085BE0D25C
:102210004FF00113C4F81C3870BD00001D4B03EBD8
:1022200080022DE9F043D2F80CC05D6DDCF814207B
:10223000461CD2F800E005EB063605EB4018516865
:1022400071450AD3D5F83438012202FA00F023EAA6
:102250000000C5F83408BDE8F083BCF81040AEEBD0
:102260000103A34228BF2346D8F81849A4B2B3EB10
:10227000840FF0D89468A4F1040959F8047F3760FA
:10228000A4EB09071F44042FF7D81C440B449460A7
:102290005360D4E7AC2C0020890141F0200101619A
:1022A00003699B06FCD41220FFF7EABA10B5054C6F
:1022B0002046FEF78DFF4FF0A0436365024BA365F8
:1022C00010BD00BFAC2C0020EC35000870B50378C1
:1022D000012B054650D12A4B446D98421BD1294B06
:1022E0005A6B42F080025A635A6D42F080025A657E
:1022F0005A6D5A6942F080025A615A6922F080028E
:102300005A610E2143205B6900F0D4FB1E4BE36051
:102310001E4BC4F800380023C4F8003EC0232360DD
:102320006E6D4FF40413A3633369002BFCDA0123B1
:1023300033610C20FFF7A4FA3369DB07FCD41220C9
:10234000FFF79EFA3369002BFCDA0026A6602846C8
:10235000FFF738FF6B68C4F81068DB68C4F81468CE
:10236000C4F81C684BB90A4BA3614FF0FF3363619B
:10237000A36843F00103A36070BD064BF4E700BF00
:10238000AC2C002000380240401400400300200222
:10239000003C30C0083C30C0F8B5446D0546002113
:1023A0002046FFF779FFA96D00234FF001128F68D7
:1023B000C4F834384FF00066C4F81C284FF0FF30E2
:1023C00004EB431201339F42C2F80069C2F8006B6C
:1023D000C2F80809C2F8080BF2D20B686A6DEB6507
:1023E000636210231361166916F01006FBD11220E8
:1023F000FFF746FAD4F8003823F4FE63C4F8003837
:10240000A36943F4402343F01003A3610923C4F8F4
:102410001038C4F814380A4BEB604FF0C043C4F8CE
:10242000103B084BC4F8003BC4F81069C4F80039ED
:10243000EB6D03F1100243F48013EA65A362F8BD6B
:10244000C835000840800010426D90F84E10D2F858
:10245000003823F4FE6343EA0113C2F800387047E2
:102460002DE9F84300EB8103456DDA68166806F044
:102470000306731E022B05EB41130C4680460FFA30
:1024800081F94FEA41104FF00001C3F8101B4FF0E3
:10249000010104F1100398BFB60401FA03F3916936
:1024A0008EBF334E06F1805606F5004600293AD01D
:1024B000578A04F15801490137436F50D5F81C1869
:1024C0000B43C5F81C382B180021C3F810195369A9
:1024D0000127611EA7409BB3138A928B9B08012A98
:1024E00088BF5343D8F85C20981842EA034301F1AF
:1024F000400205EB8202C8F85C0021465360284682
:10250000FFF7CAFE08EB8900C3681B8A43EA8453BD
:10251000483464011E432E51D5F81C381F43C5F8BA
:102520001C78BDE8F88305EB4917D7F8001B21F4A8
:102530000041C7F8001BD5F81C1821EA0303C0E7C7
:1025400004F13F0305EB83030A4A5A6028462146FB
:10255000FFF7A2FE05EB4910D0F8003923F4004341
:10256000C0F80039D5F81C3823EA0707D7E700BFC1
:102570000080001000040002826D1268C265FFF73F
:1025800021BE00005831436D49015B5813F40040EF
:1025900004D013F4001F0CBF02200120704700007C
:1025A0004831436D49015B5813F4004004D013F4E3
:1025B000001F0CBF022001207047000000EB8101CA
:1025C000CB68196A0B6813604B6853607047000052
:1025D00000EB810330B5DD68AA691368D36019B9CF
:1025E000402B84BF402313606B8A1468426D1C44E7
:1025F000013CB4FBF3F46343033323F0030302EB26
:10260000411043EAC44343F0C043C0F8103B2B6879
:1026100003F00303012B09B20ED1D2F8083802EB04
:10262000411013F4807FD0F8003B14BF43F0805377
:1026300043F00053C0F8003B02EB4112D2F8003BDC
:1026400043F00443C2F8003B30BD00002DE9F041E7
:10265000244D6E6D06EB40130446D3F8087BC3F897
:10266000087B38070AD5D6F81438190706D505EBC4
:1026700084032146DB6828465B689847FA071FD524
:10268000D6F81438DB071BD505EB8403D968CCB921
:102690008B69488A5A68B2FBF0F600FB16228AB9A9
:1026A0001868DA6890420DD2121AC3E90024202378
:1026B00083F311880B482146FFF78AFF84F31188C2
:1026C000BDE8F081012303FA04F26B8923EA0203D7
:1026D0006B81CB68002BF3D021460248BDE8F04166
:1026E000184700BFAC2C002000EB810370B5DD68FB
:1026F000436D6C692668E6604A0156BB1A444FF484
:102700000020C2F810092A6802F00302012A0AB266
:102710000ED1D3F8080803EB421410F4807FD4F8EC
:10272000000914BF40F0805040F00050C4F8000988
:1027300003EB4212D2F8000940F00440C2F800094D
:10274000D3F83408012202FA01F10143C3F8341826
:1027500070BD19B9402E84BF4020206020682E8AA9
:102760008419013CB4FBF6F440EAC44040F0005048
:102770001A44C6E7F8B504461E48456D05EB4413F8
:10278000D3F80869C3F80869F10717D5D5F81038E8
:10279000DA0713D500EB8403D9684B691F68DA6840
:1027A000974218D2D21B00271A605F60202383F360
:1027B00011882146FFF798FF87F31188330617D554
:1027C000D5F834280123A340134211D02046BDE898
:1027D000F840FFF723BD012303FA04F2038923EA3B
:1027E000020303818B68002BE8D021469847E5E778
:1027F000F8BD00BFAC2C00202DE9F74F984C666D5A
:102800007569B3691D4015F48058756107D020467D
:10281000FEF744FD03B0BDE8F04FFFF785BC002D87
:1028200012DAD6F8003E8E489F071EBFD6F8003E4B
:1028300023F00303C6F8003ED6F8043823F0010362
:10284000C6F80438FEF752FD280505D58448FFF781
:10285000B9FC8348FEF73AFDA9040CD5D6F8083830
:1028600013F0060FF36823F470530CBF43F41053B6
:1028700043F4A053F3602A0704D56368DB680BB107
:1028800077489847EB0274D4AF0227D5D4F8549018
:10289000DFF8CCB100274FF0010A09EB4712D2F85C
:1028A000003B03F44023B3F5802F11D1D2F8003B55
:1028B000002B0DDA62890AFA07F322EA0303638127
:1028C00004EB8703DB68DB6813B139465846984749
:1028D000A36D01379B68FFB29F42DED9E80617D58A
:1028E000676D3A6AC2F30A1002F00F0302F4F012A5
:1028F000B2F5802F00F08880B2F5402F08D104EBAC
:1029000083030022DB681B6A07F5805790426DD174
:102910002903D6F8184813D5E20302D50020FFF7A3
:1029200095FEA30302D50120FFF790FE670302D5B1
:102930000220FFF78BFE260302D50320FFF786FE59
:102940006D037FF567AFE00702D50020FFF712FFA8
:10295000A10702D50120FFF70DFF620702D5022073
:10296000FFF708FF23077FF555AF0320FFF702FFAE
:1029700050E7636DDFF8E8B0019300274FF0010ADC
:10298000A36D9B685FFA87F999453FF67DAF019B80
:1029900003EB4913D3F8002902F44022B2F5802F4B
:1029A00022D1D3F80029002A1EDAD3F8002942F0F8
:1029B0009042C3F80029D3F80029002AFBDB606DA0
:1029C0004946FFF769FC22890AFA09F322EA030360
:1029D000238104EB8903DB689B6813B149465846A1
:1029E00098474846FFF71AFC0137C9E7910708BF27
:1029F000D7F80080072A98BF03F8018B02F1010283
:102A000098BF4FEA182881E7023304EB830207F5E9
:102A100080575268D2F818C0DCF80820DCE9001CA6
:102A2000A1EB0C0C002188420AD104EB83046368FB
:102A30009B699A6802449A605A6802445A6067E740
:102A400011F0030F08BFD7F800808C4588BF02F84B
:102A5000018B01F1010188BF4FEA1828E3E700BFAD
:102A6000AC2C0020436D03EB4111D1F8003B43F443
:102A70000013C1F8003B7047436D03EB4111D1F8DF
:102A8000003943F40013C1F800397047436D03EB7C
:102A90004111D1F8003B23F40013C1F8003B70470B
:102AA000436D03EB4111D1F8003923F40013C1F851
:102AB0000039704700F1604303F561430901C9B271
:102AC00083F80013012200F01F039A4043099B0082
:102AD00003F1604303F56143C3F880211A60704736
:102AE00030B5039C0172043304FB0325C0E906538F
:102AF000049B03630021059BC160C0E90000C0E99D
:102B00000422C0E90842C0E90A11436330BD000055
:102B1000416A0022C0E90411C0E90A22C2606FF0D4
:102B20000101FEF71DBF0000D0E90432934201D13C
:102B3000C2680AB9181D7047002070470369196000
:102B4000C2680132C260C269134482690361934260
:102B500024BF436A03610021FEF7F6BE38B5044680
:102B60000D46E3683BB16269131D1268A36213440A
:102B7000E362002007E0237A33B929462046FEF7B6
:102B8000D3FE0028EDDA38BD6FF00100FBE700004E
:102B9000C368C269013BC3604369134482694361EE
:102BA000934224BF436A436100238362036B03B1F2
:102BB0001847704770B52023044683F31188866A4E
:102BC0003EB9FFF7CBFF054618B186F311882846BA
:102BD00070BDA36AE26A13F8015BA362934202D359
:102BE0002046FFF7D5FF002383F31188EFE70000AD
:102BF0002DE9F84F04460E46174698464FF0200937
:102C000089F311880025AA46D4F828B0BBF1000F3B
:102C100009D141462046FFF7A1FF20B18BF311886F
:102C20002846BDE8F88FD4E90A12A7EB050B521A23
:102C3000934528BF9346BBF1400F1BD9334601F1A2
:102C4000400251F8040B43F8040B9142F9D1A36AF6
:102C500040334036A3624035D4E90A239A4202D376
:102C60002046FFF795FF8AF31188BD42D8D289F339
:102C70001188C9E730465A46FEF70CF8A36A5B4450
:102C80005E44A3625D44E7E710B5029C0172043321
:102C900004FB0321C0E906130023C0E90A33039BA8
:102CA0000363049BC460C0E90000C0E90422C0E9DA
:102CB0000842436310BD0000026AC260426AC0E974
:102CC00004220022C0E90A226FF00101FEF748BE8B
:102CD000D0E904239A4201D1C26822B9184650F8BB
:102CE000043B0B607047002070470000C368C26956
:102CF0000133C3604369134482694361934224BF33
:102D0000436A43610021FEF71FBE000038B5044648
:102D10000D46E3683BB123691A1DA262E2691344C0
:102D2000E362002007E0237A33B929462046FEF704
:102D3000FBFD0028EDDA38BD6FF00100FBE7000075
:102D400003691960C268013AC260C26913448269AA
:102D50000361934224BF436A036100238362036BD0
:102D600003B118477047000070B520230D46044694
:102D7000114683F31188866A2EB9FFF7C7FF10B199
:102D800086F3118870BDA36A1D70A36AE26A0133DD
:102D90009342A36204D3E16920460439FFF7D0FFD0
:102DA000002080F31188EDE72DE9F84F04460D4629
:102DB000904699464FF0200A8AF311880026B346C0
:102DC000A76A4FB949462046FFF7A0FF20B187F315
:102DD00011883046BDE8F88FD4E90A073A1AA8EB03
:102DE0000607974228BF1746402F1BD905F140031D
:102DF00055F8042B40F8042B9D42F9D1A36A4033C7
:102E0000A3624036D4E90A239A4204D3E1692046FA
:102E10000439FFF795FF8BF311884645D9D28AF321
:102E20001188CDE729463A46FDF734FFA36A3B44B3
:102E30003D44A3623E44E5E7D0E904239A4217D11A
:102E4000C3689BB1836A8BB1043B9B1A0ED013609D
:102E5000C368013BC360C3691A44836902619A4233
:102E600024BF436A0361002383620123184670472D
:102E70000023FBE700F088B84FF08043002258633E
:102E80001A610222DA6070474FF080430022DA6054
:102E9000704700004FF08043586370474FF0804305
:102EA000586A70474B6843608B688360CB68C36027
:102EB0000B6943614B6903628B6943620B68036072
:102EC0007047000008B5264B26481A6940F2FF11EA
:102ED0000A431A611A6922F4FF7222F001021A6190
:102EE0001A691A6B0A431A631A6D0A431A651E4A55
:102EF0001B6D1146FFF7D6FF02F11C0100F5806043
:102F0000FFF7D0FF02F1380100F58060FFF7CAFF3C
:102F100002F1540100F58060FFF7C4FF02F1700177
:102F200000F58060FFF7BEFF02F18C0100F58060C4
:102F3000FFF7B8FF02F1A80100F58060FFF7B2FFCC
:102F400002F1C40100F58060FFF7ACFF02F1E0017F
:102F500000F58060FFF7A6FFBDE8084000F09AB8D2
:102F60000038024000000240F835000808B500F0C3
:102F700007FAFEF763FCFFF78FF8BDE80840FEF79D
:102F80006BBE000070470000104B1A6C42F001024B
:102F90001A641A6E42F001021A660D4A1B6E93689B
:102FA00043F0010393604FF0804353229A624FF045
:102FB000FF32DA6200229A615A63DA605A600122B3
:102FC0005A6108211A601C20FFF774BD00380240C6
:102FD000002004E04FF0804208B51169D3680B402F
:102FE000D9B2C9439B07116107D5202383F3118808
:102FF000FEF744FC002383F3118808BD08B5FFF7F2
:10300000E9FFBDE80840FFF78FB800001F4B1A69C1
:103010006FEAC2526FEAD2521A611A69C2F3080209
:103020001A614FF0FF301A695A69586100215A69D4
:1030300059615A691A6A62F080521A621A6A02F079
:1030400080521A621A6A5A6A58625A6A59625A6AED
:103050001A6C42F080521A641A6E42F080521A665C
:103060001A6E0B4A106840F480701060186F00F4FC
:103070004070B0F5007F1EBF4FF4803018671967AD
:10308000536823F40073536000F05AB900380240CB
:1030900000700040334B4FF080521A64324A4FF4B4
:1030A000404111601A6842F001021A601A689107E3
:1030B000FCD59A6822F003029A602A4B9A6812F0B3
:1030C0000C02FBD1196801F0F90119609A601A68C5
:1030D00042F480321A601A689203FCD55A6F42F0AB
:1030E00001025A671F4B5A6F9007FCD51F4A5A605E
:1030F0001A6842F080721A601B4A53685904FCD562
:10310000184B1A689201FCD5194A9A60194B1A6833
:10311000194B9A42194B21D1194A1168194A914207
:103120001CD140F205121A60144A136803F00F0311
:10313000052BFAD10B4B9A6842F002029A609A680A
:1031400002F00C02082AFAD15A6C42F480425A6406
:103150005A6E42F480425A665B6E704740F20572C6
:10316000E1E700BF0038024000700040085440070B
:1031700000948838002004E011640020003C0240E4
:1031800000ED00E041C20F41084A08B551691368DB
:103190000B4003F00103536123B1054A13680BB1DF
:1031A00050689847BDE80840FEF7BEBF003C0140AC
:1031B000242D0020084A08B5516913680B4003F01C
:1031C0000203536123B1054A93680BB1D068984755
:1031D000BDE80840FEF7A8BF003C0140242D0020B8
:1031E000084A08B5516913680B4003F004035361A2
:1031F00023B1054A13690BB150699847BDE80840EF
:10320000FEF792BF003C0140242D0020084A08B57B
:10321000516913680B4003F00803536123B1054A59
:1032200093690BB1D0699847BDE80840FEF77CBFB1
:10323000003C0140242D0020084A08B5516913685C
:103240000B4003F01003536123B1054A136A0BB11D
:10325000506A9847BDE80840FEF766BF003C014051
:10326000242D0020174B10B55A691C68144004F433
:1032700078725A61A30604D5134A936A0BB1D06AD7
:103280009847600604D5104A136B0BB1506B9847F2
:10329000210604D50C4A936B0BB1D06B9847E2051D
:1032A00004D5094A136C0BB1506C9847A30504D59B
:1032B000054A936C0BB1D06C9847BDE81040FEF7FF
:1032C00033BF00BF003C0140242D00201A4B10B535
:1032D0005A691C68144004F47C425A61620504D5A2
:1032E000164A136D0BB1506D9847230504D5134A48
:1032F000936D0BB1D06D9847E00404D50F4A136E5F
:103300000BB1506E9847A10404D50C4A936E0BB1D3
:10331000D06E9847620404D5084A136F0BB1506F02
:103320009847230404D5054A936F0BB1D06F984793
:10333000BDE81040FEF7F8BE003C0140242D0020FF
:10334000062108B50846FFF7B5FB06210720FFF761
:10335000B1FB06210820FFF7ADFB06210920FFF78E
:10336000A9FB06210A20FFF7A5FB06211720FFF77E
:10337000A1FBBDE8084006212820FFF79BBB000009
:1033800008B5FFF743FE00F00BF8FDF71FFFFDF750
:10339000F7FDFFF7F7FDBDE80840FFF76BBD000044
:1033A0000023054A19460133102BC2E9001102F12E
:1033B0000802F8D1704700BF242D0020034611F801
:1033C000012B03F8012B002AF9D1704753544D33D8
:1033D00032463F3F3F00000053544D3332463430B5
:1033E000780053544D3332463432780053544D33C1
:1033F000324634343658580000000000CC33000800
:103400003F00000013040000D83300083F00000014
:1034100019040000E23300083F000000210400000E
:10342000EC3300083F00000000000000FD0E000823
:10343000E90E0008250F0008110F00081D0F0008F5
:10344000090F0008F50E0008E10E0008310F000812
:103450000000000001000000000000006D61696EC6
:103460000000000069646C6500000000643400081E
:10347000D823002050250020010000003918000842
:10348000000000004172647550696C6F7400254241
:103490004F415244252D424C002553455249414C41
:1034A00025000000020000000000000019110008C3
:1034B0008511000840004000E8290020F82900207C
:1034C00002000000000000000300000000000000F7
:1034D000C91100080000000010000000082A0020A8
:1034E000000000000100000000000000AC2C0020E3
:1034F00001010200F51B0008051B0008A11B0008C4
:10350000851B0008430000000C3500080902430039
:10351000020100C03209040000010202010005247A
:103520000010010524010001042402020524060004
:1035300001070582030800FF09040100020A0000D8
:10354000000705010240000007058102400000005D
:10355000120000005835000812011001020000405E
:10356000091241570002010203010000040309048B
:1035700025424F41524425007265766F2D6D696E6C
:10358000692D736400303132333435363738394180
:103590004243444546000000004000000040000057
:1035A0000040000000400000000001000000020098
:1035B0000000020000000200000002000000020003
:1035C00000000200000002000000000001130008DB
:1035D000B915000865160008400040000C2D0020B9
:1035E0000C2D0020010000001C2D00208000000098
:1035F0004001000003000000000180020000000004
:10360000AAAAAAAA00010000FFFF00000000000013
:1036100000A00A004005000000000000AAAAAAAA13
:1036200040000000CFFF000000000000000000008C
:103630000000000000000000AAAAAAAA00000000E2
:10364000FFFF00000000000000000000000000007C
:1036500000000000AAAAAAAA00000000FFFF0000C4
:10366000000000000000000000000000000000005A
:10367000AAAAAAAA00000000FFFF000000000000A4
:10368000000000000000000000000000AAAAAAAA92
:1036900000000000FFFF000000000000000000002C
:1036A0000000000000000000AAAAAAAA0000000072
:1036B000FFFF00000000000000000000000000000C
:1036C000000000000A0000000000000003000000ED
:1036D00000000000000000000000000000000000EA
:1036E00000000000000000000000000000000000DA
:1036F00000000000000000007C000000000000004E
:1037000000000F0000000000FF009600000000080D
:103710000096000000000800040000006C3500085E
:103720000000000000000000000000000000000099
:08373000000000000000000091
:00000001FF
